S01A000064656D6F70726F675F73746D33326C3437362E7372656388
S31508002800F8040020914B0008CD4B0008D14B000876
S31508002810D54B0008D94B0008DD4B00080000000026
S31508002820000000000000000000000000E14B000866
S31508002830E54B000800000000E94B00086F4500085A
S31508002840ED4B0008F14B0008F54B0008F94B000862
S31508002850FD4B0008014C0008054C0008094C00080F
S315080028600D4C0008114C0008154C0008194C0008BE
S315080028701D4C0008214C0008254C0008294C00086E
S315080028802D4C0008314C0008354C0008394C00081E
S315080028903D4C0008414C0008454C0008494C0008CE
S315080028A04D4C0008514C0008554C0008594C00087E
S315080028B05D4C0008614C0008654C0008694C00082E
S315080028C06D4C0008714C0008754C0008794C0008DE
S315080028D07D4C0008814C0008854C0008894C00088E
S315080028E08D4C0008914C0008954C0008994C00083E
S315080028F09D4C0008A14C0008A54C0008A94C0008EE
S31508002900AD4C0008B14C0008B54C0008B94C00089D
S31508002910BD4C0008C14C0008C54C0008C94C00084D
S31508002920CD4C0008D14C0008D54C0008D94C0008FD
S31508002930DD4C0008E14C0008E54C0008E94C0008AD
S31508002940ED4C0008F14C0008F54C0008F94C00085D
S31508002950FD4C0008014D0008054D0008094D00080A
S315080029600D4D0008114D0008154D0008194D0008B9
S315080029701D4D0008214D0008254D000800000000E7
S31508002980294D00082D4D0008EE11AA552DE9FC41E8
S31508002990040000202078C00649D5DFF83458286896
S315080029A010F00C0F40F08080DFF820683068800750
S315080029B004D5A069002801D101206EE2306800071D
S315080029C003D5306810F0F00005E0DFF8100800685D
S315080029D0000910F0F000216A88424BD2206A00F004
S315080029E0B5FB002801D0012057E2306850F00800F6
S315080029F03060316831F0F001206A01433160DFF858
S31508002A00E007016831F47F41E26951EA0221016079
S31508002A1000F01BFBDFF8CC172A68C2F30312895CA7
S31508002A20C840DFF8B0170860002000F0EFFB2078F8
S31508002A30C00740F1BB80DFF89807016811F00C0168
S31508002A4008290BD0006810F00C000C2869D1DFF8B3
S31508002A508807006810F00300032862D1DFF86C07C6
S31508002A600068800340F1A2806068002840F09E80DC
S31508002A70012012E2306850F008003060316831F009
S31508002A80F001206A01433160DFF85407016831F428
S31508002A907F41E26951EA02210160206A00F056FB93
S31508002AA00028B5D00120F8E1A069002826D0DFF873
S31508002AB01C57286850F00100286000F0BBFB060090
S31508002AC02868800706D400F0B5FB801B0328F7D3D7
S31508002AD00320E2E1286850F008002860296831F0F0
S31508002AE0F001206A01432960DFF8F406016831F431
S31508002AF07F41E26951EA0221016098E7DFF8CC6676
S31508002B00306840084000306000F094FB05003068EB
S31508002B1080078CD500F08EFB401B0328F7D30320D3
S31508002B20BBE16068B0F5803F06D1DFF8A006016812
S31508002B3051F48031016018E06068B0F5A02F0AD121
S31508002B40DFF88806016851F480210160016851F4B4
S31508002B508031016009E0DFF87406016831F48031DC
S31508002B600160016831F480210160606800280ED098
S31508002B7000F060FB0500DFF854060068800315D4F2
S31508002B8000F058FB401B6528F5D3032085E100F0CB
S31508002B9051FB0500DFF834060068800306D500F00F
S31508002BA049FB401B6528F5D3032076E1207880078A
S31508002BB025D5DFF81C06016811F00C0104290BD095
S31508002BC0006810F00C000C2832D1DFF80C060068FB
S31508002BD010F0030002282BD1DFF8F0050068400545
S31508002BE004D5E068002801D1012056E1DFF8F00598
S31508002BF0016831F0F851226951EA026101602078D2
S31508002C0000075BD56069002845D0DFF8D0653068D5
S31508002C1050F00100306000F00DFB050030688007B9
S31508002C204CD400F007FB401B0328F7D3032034E1FC
S31508002C30E06800281CD0DFF89465306850F480708E
S31508002C40306000F0F7FA05003068400506D400F059
S31508002C50F1FA401B0328F7D303201EE1DFF88005AD
S31508002C60016831F0F851226951EA02610160C6E74C
S31508002C70DFF85865306830F48070306000F0DAFAB2
S31508002C80050030684005BAD500F0D4FA401B032881
S31508002C90F7D3032001E1DFF84465306840084000B7
S31508002CA0306000F0C7FA05003068800706D500F0E6
S31508002CB0C1FA401B0328F7D30320EEE0207840072B
S31508002CC074D50026DFF820552868C00009D428687E
S31508002CD050F080502860286810F0805000900098C6
S31508002CE00126DFF808753868C00511D4386850F42D
S31508002CF08070386000F09EFA80463868C00507D4B0
S31508002D0000F098FAB0EB08000328F6D30320C4E0D5
S31508002D10A068012806D1DFF8D804016851F001013E
S31508002D20016017E0A06805280AD1DFF8C404016825
S31508002D3051F004010160016851F00101016009E0E8
S31508002D40DFF8AC040168490849000160016831F000
S31508002D5004010160A068002810D000F06BFA070093
S31508002D60DFF88C040068800719D400F063FAC01BEA
S31508002D7041F289318842F3D303208EE000F05AFAF3
S31508002D800700DFF86C040068800708D500F052FADF
S31508002D90C01B41F289318842F3D303207DE0F6B2A5
S31508002DA0012E03D1286830F080502860A06A0028D8
S31508002DB072D0DFF81C04006810F00C000C2869D0EB
S31508002DC0A06A022840D1DFF80454286830F08070E1
S31508002DD0286000F02FFA06002868800106D500F062
S31508002DE029FA801B0328F7D3032056E0DFF8E813F7
S31508002DF0206B401E626B120252EA0012A06B000999
S31508002E0052EA4042E06A0243E06B4008401E52EA3A
S31508002E104052206C4008401E52EA40620A60286808
S31508002E2050F080702860086850F08070086000F0E4
S31508002E3001FA0400286880012ED400F0FBF9001B73
S31508002E400328F7D3032028E0DFF88043206830F012
S31508002E50807020602068000108D42068800005D4AE
S31508002E60DFF874030168890889000160DFF86813D0
S31508002E700A68DFF8800302400A6000F0DBF9050003
S31508002E802068800108D500F0D5F9401B0328F7D340
S31508002E90032002E0012000E00020BDE8F6812DE9CC
S31508002EA0F04104000D000020DFF84C63306810F094
S31508002EB00700A8420BD23068C008C000284330601B
S31508002EC0306810F00700A84201D00120BBE0207846
S31508002ED0C00773D56068032806D1DFF8F0020068DA
S31508002EE080011CD40120AEE06068022806D1DFF814
S31508002EF0DC020068800312D40120A4E06068002880
S31508002F0006D1DFF8C8020068800708D401209AE0D5
S31508002F10DFF8B8020068400501D4012093E0DFF825
S31508002F20B07239688908890060680143396000F021
S31508002F3081F98046606803280ED1386810F00C00C5
S31508002F400C283BD000F076F9B0EB080041F2893145
S31508002F508842F2D3032076E0606802280ED13868EA
S31508002F6010F00C00082829D000F064F9B0EB08002E
S31508002F7041F289318842F2D3032064E06068002870
S31508002F800DD1386810F00C0F18D000F053F9B0EBDB
S31508002F90080041F289318842F3D3032053E03868A8
S31508002FA010F00C00042809D000F044F9B0EB080032
S31508002FB041F289318842F2D3032044E02078800721
S31508002FC007D5DFF80C120A6832F0F002A06802434F
S31508002FD00A60306810F0070085420BD23068C008D6
S31508002FE0C00028433060306810F00700A84201D0BE
S31508002FF0012028E02078400707D5DFF8D4110A68B1
S3150800300032F4E062E06802430A602078000708D5D7
S31508003010DFF8BC01016831F46051226951EAC20146
S31508003020016000F012F8DFF8BC11DFF8A42112687D
S31508003030C2F30312895CC840DFF8981108600020C3
S3150800304000F0E4F80020BDE8F0810022002000200E
S315080030500220022000205E490B6813F00C0F0AD0EC
S315080030600B6813F00C030C2B1AD15B4B1B6813F07F
S315080030700303012B14D1554A13681B0704D4574A76
S315080030801268C2F3032202E01268C2F303125B4B12
S3150800309053F822200B6813F00C0F0ED110000CE029
S315080030A00B6813F00C03042B01D1554805E00B6897
S315080030B013F00C03082B00D15248096811F00C01D3
S315080030C00C2929D1444B186810F003001968C1F37C
S315080030D00211491C022802D0032808D00FE04848EC
S315080030E0B0FBF1F11868C0F3062041430DE04548EE
S315080030F0B0FBF1F11868C0F30620414305E0B2FBC6
S31508003100F1F11868C0F3062041431868C0F341601E
S31508003110401C4000B1FBF0F070472E48006870472D
S3150800312080B5FFF7FAFF3849294A1268C2F3022226
S31508003130895CC84002BD80B5FFF7EFFF3249244AD3
S315080031401268C2F3C222895CC84002BD7CB504007D
S3150800315000200025244E3068C00002D500F070F823
S315080031600EE0306850F080503060306810F08050C3
S315080031700090009800F064F8316831F080513160B1
S31508003180B0F5007F07D1812C10D3A12C01D30225DD
S315080031900CE001250AE0812C01D3032506E0802CEA
S315080031A001D1022502E0702C00D1012512480168E0
S315080031B0C908C90029430160006810F00700A84241
S315080031C001D0012000E0002076BD0000001002407A
S315080031D008100240000000200C1002409410024023
S315080031E004100240A84B0008581002400070004026
S315080031F090100240FFFFEEFE00200240844A0008BD
S315080032000024F40000127A00C44B000810B504002C
S31508003210074800684FF47A71B0FBF1F000F0C8F87F
S31508003220002221005FF0FF3000F0B1F8002010BD49
S315080032300000002001480068704700BFF000002029
S31508003240DFF88000006810F4C06070470021B0F510
S31508003250007F26D1DFF86C00016811F4C061B1F572
S31508003260007F2CD0016831F4C06151F4007101600F
S31508003270DFF854000068DFF85410B0FBF1F0322193
S31508003280484300E0401E002804D0DFF844100968CF
S315080032904905F7D4DFF83800006840050FD5032044
S315080032A00EE0DFF82000016811F4C061B1F5806F07
S315080032B005D0016831F4C06151F4806101600020D5
S315080032C070470000007000400000002040420F00D8
S315080032D01470004010F00700404B1A684FF6FF01C3
S315080032E00A403F4951EA00210A431A6070473B48A1
S315080032F00068C0F302207047020052B2002A08D5BF
S315080033000901384A40B210F00F00104400F8041CB6
S3150800331003E00901344A40B21154704710B410F062
S315080033200700D0F10703052B01D3042301E0D0F1F0
S315080033300703041D072C01D2002000E0C01E01244B
S3150800334014FA03F35B1E1940814014FA00F0401E7C
S315080033501040084310BC704780B5411EB1F1807F0C
S3150800336001D301200EE0401E204908600F215FF0BE
S31508003370FF30FFF7C1FF00201D49086007201D49DF
S315080033800860002002BD80B5FFF7A4FF01BD70B537
S3150800339004000D0016000020FFF7A9FF32002900DF
S315080033A0FFF7BCFF0100200040B2FFF7A5FF70BD84
S315080033B080B5FFF7D1FF02BD042805D10D48016885
S315080033C051F00401016004E00A48016831F0040183
S315080033D00160704780B500F00FF801BD0CED00E004
S315080033E00000FA0518ED00E000E400E014E000E053
S315080033F018E000E010E000E0704730B4002513E064
S3150800340050F8042BD30744BFA9F101039A18091FE2
S31508003410042942F8045BFAD213468C0744BF158088
S315080034209B1CC90748BF1D7050F8041B0029E7D12B
S3150800343030BC704710B50400002C01D1012037E0DC
S31508003440A0690028FFD194F87100002805D1002052
S3150800345084F87000200000F0A2FB242084F8710094
S31508003460206800684008400021680860200000F0D5
S31508003470ABF8012801D101201AE0606A002802D0C1
S31508003480200000F0B1FA2068406830F490402168C6
S3150800349048602068806830F02A00216888602068C3
S315080034A0006850F0010021680860200000F009FB60
S315080034B010BD2DE9FC4105000C0090461E000020B9
S315080034C095F8720020287CD1002C03D0404680B2A3
S315080034D0002801D1012075E095F87000012801D176
S315080034E002206FE0012085F870000020686722201E
S315080034F085F87200FFF79EFE0700A5F85880A5F824
S315080035005A80A868B0F5805F0BD12869002804D1D5
S3150800351040F2FF10A5F85C001FE0FF20A5F85C004C
S315080035201BE0A86800280AD12869002803D1FF20D3
S31508003530A5F85C0011E07F20A5F85C000DE0A868FE
S31508003540B0F1805F09D12869002803D17F20A5F84A
S315080035505C0002E03F20A5F85C00B5F85C8019E045
S315080035602868808C18EA00002070641C0DE0A868A2
S31508003570B0F5805FF4D128690028F1D120002968C8
S31508003580898C18EA01010180A41CB5F85A00401E6E
S31508003590A5F85A00B5F85A0000280AD000963B004C
S315080035A000222021280000F0C3FA0028DFD00320DB
S315080035B008E0202085F87200002085F870000020B9
S315080035C000E00220BDE8F681F8B5040000201027C7
S315080035D00020002600250020DFF8DC232168914220
S315080035E0FFD0A36821690B4361690B43E1690B436B
S315080035F02168D1F800C0DFF8C41311EA0C0C53EAAD
S315080036000C0321680B6021684B6833F44053E1686A
S315080036100B4321684B60A3692168914201D0216A56
S315080036200B432168896831F430610B4321688B604C
S315080036302168DFF88C33994216D1DFF888130968B8
S3150800364011F00301002905D0022905D006D3032964
S3150800365006D007E0012798E0022796E0042794E0C1
S31508003660082792E0102790E02168DFF85C3399423A
S3150800367017D1DFF85013096811F00C01002906D09C
S31508003680042908D0082904D00C2906D007E0002709
S315080036907BE0022779E0042777E0082775E0102702
S315080036A073E02168DFF82433994217D1DFF8141341
S315080036B0096811F03001002906D0102908D0202900
S315080036C004D0302906D007E000275EE002275CE038
S315080036D004275AE0082758E0102756E02168DFF843
S315080036E0F032994217D1DFF8DC12096811F0C001EF
S315080036F0002906D0402908D0802904D0C02906D040
S3150800370007E0002741E002273FE004273DE00827BD
S315080037103BE0102739E02168AE4B994219D1A949F7
S31508003720096811F44071002909D0B1F5807F0AD0E3
S31508003730B1F5007F05D0B1F5407F06D007E0002738
S3150800374023E0022721E004271FE008271DE01027B1
S315080037501BE02168914218D19A49096811F4406121
S31508003760002909D0B1F5806F0AD0B1F5006F05D0F0
S31508003770B1F5406F06D007E0002706E0022704E00F
S31508003780042702E0082700E010272168914270D13B
S315080037903900C9B2002906D0022907D0042907D062
S315080037A0082908D00AE0FFF7BBFC08E08A4806E0CB
S315080037B0FFF74BFC03E04FF4004000E0012500282A
S315080037C000F0F280626803214A43904205D362689A
S315080037D04FF480514A43824201D20125E4E0FFB208
S315080037E0002F06D0022F14D0042F1FD0082F2DD05B
S315080037F034E0FFF795FC02004FF4807360684008D8
S315080038000021E3FB02016268002300F0C9F9060003
S3150800381025E0606840080021704A00238018594155
S315080038206268002300F0BCF9060018E0FFF70DFCFB
S3150800383002004FF48073606840080021E3FB020130
S315080038406268002300F0ACF9060008E060684008EA
S3150800385010F500006168B0FBF1F600E00125B6F549
S3150800386040705F49884202D22068C6609CE0012504
S315080038709AE0E069B0F5004F4FD1FFB2002F08D0AB
S31508003880012F11D0022F1AD0042F21D0082F2AD0A9
S3150800389032E0FFF745FC6168490811EB40016068B2
S315080038A0B1FBF0F6B6B228E0FFF745FC61684908B7
S315080038B011EB40016068B1FBF0F6B6B21DE0606836
S315080038C0484911EB50016068B1FBF0F6B6B214E056
S315080038D0FFF7BBFB6168490811EB40016068B1FB63
S315080038E0F0F6B6B209E06068400810F58030616805
S315080038F0B0FBF1F6B6B200E001254FF6F071B6F16D
S315080039001000884207D23140C6F34200014389B20B
S315080039102068C16048E0012546E0FFB2002F08D0C4
S31508003920012F10D0022F18D0042F1FD0082F27D010
S315080039302FE0FFF7F5FB616810EB51006168B0FBFB
S31508003940F1F6B6B226E0FFF7F6FB616810EB510018
S315080039506168B0FBF1F6B6B21CE060681E4911EB6F
S3150800396050016068B1FBF0F6B6B213E0FFF76DFBE5
S31508003970616810EB51006168B0FBF1F6B6B209E078
S315080039806068400810F500406168B0FBF1F6B6B211
S3150800399000E00125B6F110004FF6F071884202D218
S315080039A02068C66000E001250020206600206066C9
S315080039B02800C0B2F2BD000000800040F369FFEFA6
S315080039C0003801408810024000440040004800408A
S315080039D0004C0040005000400024F400000024F48D
S315080039E000FD0F000048E80190F82410C90707D524
S315080039F001684A6832F40032816A0A4301684A60FB
S31508003A0090F82410890707D501684A6832F480328D
S31508003A10C16A0A4301684A6090F82410490707D525
S31508003A2001684A6832F48022016B0A4301684A60D9
S31508003A3090F82410090707D501684A6832F400424D
S31508003A40416B0A4301684A6090F82410C90607D5F5
S31508003A5001688A6832F48052816B0A4301688A6079
S31508003A6090F82410890607D501688A6832F400524E
S31508003A70C16B0A4301688A6090F82410490613D579
S31508003A8001684A6832F48012016C0A4301684A6088
S31508003A90016CB1F5801F07D101684A6832F4C0028B
S31508003AA0416C0A4301684A6090F82410090607D554
S31508003AB001684A6832F40022816C0A430068426051
S31508003AC0704738B50400002000206067FFF7B2FB96
S31508003AD005002068006800070DD57FF07E4000903D
S31508003AE02B0000225FF40011200000F021F80028C6
S31508003AF001D003201BE02068006840070DD57FF041
S31508003B007E4000902B0000225FF48001200000F028
S31508003B100FF8002801D0032009E0202084F871005E
S31508003B20202084F87200002084F87000002032BD3E
S31508003B302DE9F04105000E0090461F00069C2868F6
S31508003B40C0693040B04201D1012000E00020414662
S31508003B50C9B2884220D114F1010FF0D0002C04D04C
S31508003B60FFF768FBC01B8442E9D22868006830F476
S31508003B70D07029680860286880684008400029686D
S31508003B808860202085F87100202085F872000020C2
S31508003B9085F87000032000E00020BDE8F08170473A
S31508003BA0BBBBE1B1B2F5803F80F07E80022A1ED908
S31508003BB08C46B1FBF2F102FB11C31B0443EA104326
S31508003BC0B3FBF2FC02FB1C3380B240EA0343B3FBAF
S31508003BD0F2F002FB103240EA0C4000237047022A3A
S31508003BE005D98446B0FBF2F002FB10C270474AB111
S31508003BF005D100F0010249085FEA3000704700224B
S31508003C000023704700F0E4B80B00020000210020F2
S31508003C107047904271EB030CF6D3B3F5803F2FD271
S31508003C20F0B5B3FA83F7B1FA81F4A7F10F0E3D1B8D
S31508003C305340CEF1200602FA0EF2F3415340B5F195
S31508003C400F0746D80F3C2C444140C4F12006A0403B
S31508003C50F1414140B1FBF3F603FB1611A2FB064501
S31508003C60001BA94102D2761E8018594180EA01023A
S31508003C7021FA0EF362FA0EF200215A403046F0BDE0
S31508003C8030B4B1FBF3FC03FB1C11A2FB0C45001B73
S31508003C90A94103D2ACF1010C8018594130BC024647
S31508003CA00B46604600217047B2F1807F65D3F0B5B8
S31508003CB0B2FA82F7B1FA81F4C7F10F063D1B22FA70
S31508003CC006F307F1110EF24120355A40B5F10F07F8
S31508003CD0B8D94140C4F12006A040F1414140B1FBAA
S31508003CE0F3FC03FB1C11A2FB0C45001BA94103D2E4
S31508003CF0BCF1010C801859410F2F12D30F3FC9038D
S31508003D0041EA5041B1FBF3F603FB1611A2FB064547
S31508003D10D4EBC030A94102D2761E8018594146EA32
S31508003D20CC3C07B34140C7F12006B840F1414140B9
S31508003D30B1FBF3F603FB1611A2FB0645001BA941CE
S31508003D4002D2761E8018594180EA010221FA0EF342
S31508003D50C7F1200462FA0EF20CFA07F05A402CFA60
S31508003D6004F13043F0BD80EA010221FA0EF3002186
S31508003D7062FA0EF260465A40F0BD8C46B1FBF2F18B
S31508003D8002FB11C31B0243EA1063B3FBF2FC02FBFE
S31508003D901C331B024CEA002043EA1063B3FBF2FC17
S31508003DA002FB1C331B024CEA002043EA1063B3FBF8
S31508003DB0F2FC02FB1C331B024CEA002043EA1063A8
S31508003DC0B3FBF2FC02FB1C324CEA002000237047CE
S31508003DD0704730B40EE00268436802440830DC07D6
S31508003DE044BFA9F10104E31852F8045B43F8045BE5
S31508003DF0091FF9D150F8041B0029ECD130BC7047D3
S31508003E0038B504000020002C01D10120AEE094F85A
S31508003E102000002802D1200000F006FA2068006879
S31508003E2030F0020021680860FFF704FA05002068F0
S31508003E30406880070DD5FFF7FDF9401B0B28F6D320
S31508003E40606A50F400306062052084F82000012082
S31508003E508CE02068006850F0010021680860FFF7D0
S31508003E60E9F9050020684068C0070DD4FFF7E2F9B4
S31508003E70401B0B28F6D3606A50F4003060620520B8
S31508003E8084F82000012071E0207E012806D12068F0
S31508003E90006850F080002168086005E02068006826
S31508003EA030F0800021680860607E012806D120680D
S31508003EB0006850F040002168086005E02068006846
S31508003EC030F0400021680860A07E012806D12068ED
S31508003ED0006850F020002168086005E02068006846
S31508003EE030F0200021680860E07E012806D12068AD
S31508003EF0006830F010002168086005E02068006856
S31508003F0050F0100021680860207F012806D120683B
S31508003F10006850F008002168086005E0206800681D
S31508003F2030F0080021680860607F012806D1206803
S31508003F30006850F004002168086005E02068006801
S31508003F4030F0040021680860A168E0680143206930
S31508003F500143606901436068401E01432068C161EE
S31508003F6000206062012084F82000002032BD30B4B1
S31508003F700022026890F82030012B03D090F82030F8
S31508003F80022B6ED1D2F8000250F00100C2F80002EE
S31508003F9001204B6910FA03F3D2F81C029843C2F8C1
S31508003FA01C02C869002816D1D2F80C029843C2F838
S31508003FB00C02486902EBC000CC684D68C5EA0444A7
S31508003FC0C0F84042486902EBC0008C680D68C5EA33
S31508003FD00444C0F84442C869012816D1D2F80C0234
S31508003FE01843C2F80C02486902EBC0000C684D6819
S31508003FF0C5EA0444C0F84042486902EBC0008C6830
S31508004000CD68C5EA0444C0F844428869002805D149
S31508004010D2F804029843C2F8040204E0D2F8040273
S315080040201843C2F804020869002805D1D2F8140218
S315080040309843C2F8140204E0D2F814021843C2F8EE
S315080040401402086A012804D1D2F81C020343C2F8F4
S315080040501C32D2F8000240084000C2F800020020D4
S3150800406004E0416A51F480214162012030BC704766
S3150800407038B50400002094F82000012821D1022038
S3150800408084F820002068006840084000216808601D
S31508004090FFF7D0F8050020684068C0070DD5FFF780
S315080040A0C9F8401B0B28F6D3606A50F400306062EA
S315080040B0052084F82000012008E000206062002026
S315080040C004E0606A50F400206062012032BD30B41A
S315080040D090F82040012C04D090F82040022C40F0A3
S315080040E09C8000290AD10468E46814F0030F12D1F1
S315080040F0416A51F400114162012093E001290AD175
S315080041000468246914F0030F05D1416A51F40011BB
S315080041104162012086E004680D012C44D4F8B041C0
S3150800412014F0040494609468002C07D104680D0107
S315080041302C44D4F8B041640D146006E004680D01FF
S315080041402C44D4F8B041E408546004680D012C44AA
S31508004150D4F8B041C4F34004D46004680D012C447B
S31508004160D4F8B44114F00F04146104680D012C440A
S31508004170D4F8B441C4F30724946104680D012C44AF
S31508004180D4F8B441240C546102680C012244D2F8D4
S31508004190B8211A7002680C012244D2F8B821120A12
S315080041A05A7002680C012244D2F8B821120C9A708F
S315080041B002680C012244D2F8B821120EDA7002689D
S315080041C00C012244D2F8BC211A7102680C0122445F
S315080041D0D2F8BC21120A5A7102680C012244D2F89C
S315080041E0BC21120C9A7102680C012244D2F8BC2137
S315080041F0120EDA71002906D10168C96851F020014A
S315080042000068C16007E0012905D10168096951F014
S31508004210200100680161002004E0416A51F4802110
S315080042204162012030BC704770470000BFF34F8FD2
S31508004230B6490A6812F4E062B54802430A60BFF359
S315080042404F8F00BFFDE780B500F00DF800F0CDF800
S3150800425001BD80B500F021F800F02AF901BD80B54E
S31508004260FFF7E4FF01BD80B5AA48AB4901604FF4EA
S3150800427061414160002181600021C1600021016126
S31508004280002181610C2141610021C1610021016287
S3150800429000214162FFF7CEF801BD70B59F4C20782A
S315080042A0002815D19E4D280000F037F8012833D193
S315080042B02878002830D0287841282DDA00F053F9DC
S315080042C0984908600120207000209749087023E06B
S315080042D0954D934E28783044401C00F01EF801286E
S315080042E011D12878401C287028783178884213D153
S315080042F0002020707078FF280ED1287802280BD16C
S31508004300FFF7ADFF08E000F02EF986490968643129
S31508004310814201D20020207070BD80B501000023C3
S3150800432001227C48FFF7C5F8C0B2002801D1012058
S3150800433000E0002002BDF8B504000D0016001F00BD
S31508004340FEF7EEFE4FF47A71B0FBF1F1002200E0C1
S31508004350521C1000C0B2122845D2744B200080B2FD
S3150800436094465FFA8CFC13F81CC096465FFA8EFEDC
S3150800437003EB4E0E9EF801E01EEB0C0C1CF1010C33
S315080043800CFB00F0B1FBF0FC00FB1C100028DFD191
S31508004390200080B294465FFA8CFC13F81CC096463F
S315080043A05FFA8EFE03EB4E0E9EF801E01EEB0C0C38
S315080043B01CF1010C0CFB00F0B1FBF0F028802888FA
S315080043C00028C5D0288840F2014C6045C0DA1000A4
S315080043D0C0B213F810003070D2B203EB4200407836
S315080043E03870012000E00020F2BD30B58BB0002007
S315080043F0ADF8020000208DF8010000208DF80000BD
S3150800440040F267656B460DF101020DF102014FF4AA
S31508004410FA70FFF790FF464C464820600020207649
S31508004420002060760020A0760020E0760020207725
S31508004430002060770020A0600020E0609DF8010061
S31508004440401E000420619DF80000401E00056061C2
S31508004450BDF8020060602000FFF7D2FC002D02D4F0
S315080044606D05354805E025F00045ED0055F00405D5
S31508004470324800210691002107910121089129005F
S31508004480090C0191ADB202950100090C039180B2A5
S31508004490049000200590012009900E200A9001A999
S315080044A02000FFF764FD2000FFF7E2FD0BB030BDEA
S315080044B030B589B040F2676400256B4602AA002130
S315080044C01B48FFF704FE00281ED1002C07D40298CB
S315080044D0A0420DD1049800280AD1012508E024F04D
S315080044E000440398A04203D10498042800D101256A
S315080044F0EDB2012D08D19DF80000FF2804D10698D9
S31508004500022801D1FFF7ABFE09B030BD0CED00E083
S315080045100400FA050400002000440040F5000020CD
S315080045207C000020E8000020F4000020DC4A000897
S31508004530C0000020006400400400E0FFFCFF1F00EC
S3150800454080B5FEF7EAFD4FF47A71B0FBF1F0FEF79D
S315080045502FFF0420FEF730FF002200215FF0FF3016
S31508004560FEF715FF01BD80B5FEF764FE02BD80B5F6
S3150800457000F004F8FEF72EFF01BD000002480168AE
S31508004580491C0160704700BFF0000020F8B4020023
S3150800459000240020002036E0072704E0DFF8F03189
S315080045A09A42F9D1062714F00303DBB29B009F4019
S315080045B03E4323009B0845F82360DFF8D8512B6853
S315080045C083434E68F60300D503432B60DFF8C851D2
S315080045D02B6883434E68B60300D503432B60DFF888
S315080045E0BC512B6883434E68F60200D503432B6003
S315080045F0DFF8AC512B6883434E68B60201D51843E1
S3150800460003002B60641C0868E040002800F0B480B2
S315080046100125086815FA04F318400028F2D04B68FB
S31508004620022B02D04B68122B17D12300DB0802EBB2
S3150800463083031E6A0F2714F00703DBB29B009F4013
S31508004640BE430F6914F00703DBB29B009F403E434D
S315080046502300DB0802EB83031E6217680326230088
S31508004660DBB25B0016FA03F39F4391F804C01CF013
S31508004670030C2300DBB25B001CFA03FC5CEA0707A9
S3150800468017604B68012B08D04B68022B05D04B6886
S31508004690112B02D04B68122B1AD197682300DBB274
S315080046A05B0016FA03F39F43D1F80CC02300DBB274
S315080046B05B001CFA03FC5CEA07079760576815FA63
S315080046C004F39F434B68C3F30013A3401F4357608B
S315080046D00B7913F00303032B08D1D36AA540AB4328
S315080046E04D68C5F3C005A5402B43D362D5682300A2
S315080046F0DBB25B009E40B5438E682300DBB25B00ED
S315080047009E403543D5604B68DB007FF57BAF254B74
S315080047101D6855F001051D601B6813F00103009321
S31508004720009B214D23009B0855F823600F2714F0A2
S315080047300303DBB29B009F40BE43B2F1904F01D109
S31508004740002730E7194B9A4201D101272BE7184B6E
S315080047509A4201D1022726E7164B9A4201D103272E
S3150800476021E7154B9A4201D104271CE7134B9A42BD
S315080047707FF414AF052716E7F1BC7047D2B2002ABA
S3150800478002D089B2816101E089B281627047000076
S3150800479000180048000401400404014008040140D0
S315080047A00C04014060100240080001400004004863
S315080047B000080048000C0048001000480014004893
S315080047C080B500F007F8FFF73EFD00F0F3F8FFF7B5
S315080047D040FDFAE780B500F009F800F011F900F09D
S315080047E009F8FFF7ADFE00F0DDF801BD6748684936
S315080047F00860704780B596B0022005904FF4807027
S3150800480008901020099002200F9002201090012095
S3150800481011900A201290072013900220149002206B
S31508004820159005A8FEF7B2F8002800D0FEE70F207D
S3150800483000900320019000200290002003900020A1
S31508004840049003216846FEF72AFB002800D0FEE7FD
S315080048504FF40070FEF7FAFC002800D0FEE717B008
S3150800486000BD80B586B04B48016851F00101016072
S31508004870006810F00100059005984748016851F056
S3150800488080510160016811F08051059105994349ED
S315080048900A6852F001020A600A6812F001020592DB
S315080048A0059A0A6852F002020A60096811F00201C4
S315080048B005910599016851F400310160016811F408
S315080048C0003105910599016851F000710160006891
S315080048D010F00070059005980320FEF754FD00229D
S315080048E000217FF00B00FEF752FD002200217FF029
S315080048F00A00FEF74CFD002200217FF00900FEF7B2
S3150800490046FD002200217FF00400FEF740FD00224C
S3150800491000217FF00300FEF73AFD002200217FF018
S315080049200100FEF734FD002200215FF0FF30FEF79C
S315080049302EFD2020009001200190002002900020EA
S31508004940039069465FF09040FFF720FE0C20009028
S315080049500220019000200290032003900720049073
S3150800496069465FF09040FFF711FE4FF440700090E3
S315080049700220019000200290032003900920049051
S3150800498069460748FFF702FE07B000BD0028000881
S3150800499008ED00E060100240581002404C1002403A
S315080049A00004004880B5002220215FF09040FFF700
S315080049B0E5FE01BD38B5FFF7D6FD04000E4D2868A3
S315080049C0201AB0F5FA7F15D30C490878002808D1C3
S315080049D001200870012220215FF09040FFF7CEFEEB
S315080049E007E000200870002220215FF09040FFF7C2
S315080049F0C5FE2C6031BD0000EC000020F60000204A
S31508004A0080B50748016851F4807101600320FEF7FC
S31508004A10BAFC0020FEF7FAFBFFF723FF002002BDD1
S31508004A20002002401048016851F4700101600F49E6
S31508004A30086850F00100086000200D4A10600A68F6
S31508004A400C4802400A604FF480500B4A1060086810
S31508004A5030F4802008600020084908605FF0006094
S31508004A60074908607047000088ED00E00010024022
S31508004A7008100240FFFFF6EA0C1002401810024028
S31508004A8008ED00E0A0860100400D0300801A06002C
S31508004A9000350C0040420F0080841E0000093D00CE
S31508004AA000127A000024F40000366E010048E8017E
S31508004AB0006CDC0210B5074979441831064C7C4471
S31508004AC0163404E00A68081D114488470146A142C5
S31508004AD0F8D110BD50000000700000000502060263
S31508004AE0060307030803090309040A040B040C0454
S31508004AF00C050D050E050F050F0610061007100804
S31508004B004EF68851CEF20001086840F4700008603D
S31508004B10BFF34F8FBFF36F8F4FF00070E1EE100AAF
S31508004B2070470000D7E8FFFFF400000004000020EB
S31508004B30000000009FF2FFFF04000000F4010000DF
S31508004B40000000200000000000F00DF8002801D049
S31508004B50FFF7B0FFAFF300800020AFF30080FFF748
S31508004B602FFE00F002F80120704700F001B800009F
S31508004B700746384600F002F8FBE7000080B5AFF3B9
S31508004B800080024A11001820ABBEFBE7260002008F
S31508004B90024885460248804702480047F804002034
S31508004BA0254A0008B94B0008000000000000000074
S31508004BB00102030406070809AFF30080FFF7A0FF08
S31508004BC0FFF7C2FF0000000001020304FFF7FEBF63
S31508004BD0FFF7FEBFFFF7FEBFFFF7FEBFFFF7FEBFFB
S31508004BE0FFF7FEBFFFF7FEBFFFF7FEBFFFF7FEBFEB
S31508004BF0FFF7FEBFFFF7FEBFFFF7FEBFFFF7FEBFDB
S31508004C00FFF7FEBFFFF7FEBFFFF7FEBFFFF7FEBFCA
S31508004C10FFF7FEBFFFF7FEBFFFF7FEBFFFF7FEBFBA
S31508004C20FFF7FEBFFFF7FEBFFFF7FEBFFFF7FEBFAA
S31508004C30FFF7FEBFFFF7FEBFFFF7FEBFFFF7FEBF9A
S31508004C40FFF7FEBFFFF7FEBFFFF7FEBFFFF7FEBF8A
S31508004C50FFF7FEBFFFF7FEBFFFF7FEBFFFF7FEBF7A
S31508004C60FFF7FEBFFFF7FEBFFFF7FEBFFFF7FEBF6A
S31508004C70FFF7FEBFFFF7FEBFFFF7FEBFFFF7FEBF5A
S31508004C80FFF7FEBFFFF7FEBFFFF7FEBFFFF7FEBF4A
S31508004C90FFF7FEBFFFF7FEBFFFF7FEBFFFF7FEBF3A
S31508004CA0FFF7FEBFFFF7FEBFFFF7FEBFFFF7FEBF2A
S31508004CB0FFF7FEBFFFF7FEBFFFF7FEBFFFF7FEBF1A
S31508004CC0FFF7FEBFFFF7FEBFFFF7FEBFFFF7FEBF0A
S31508004CD0FFF7FEBFFFF7FEBFFFF7FEBFFFF7FEBFFA
S31508004CE0FFF7FEBFFFF7FEBFFFF7FEBFFFF7FEBFEA
S31508004CF0FFF7FEBFFFF7FEBFFFF7FEBFFFF7FEBFDA
S31508004D00FFF7FEBFFFF7FEBFFFF7FEBFFFF7FEBFC9
S31508004D10FFF7FEBFFFF7FEBFFFF7FEBFFFF7FEBFB9
S31508004D20FFF7FEBFFFF7FEBFFFF7FEBFFFF7FEBFA9
S30908004D3000093D002B
S70508004BB9EE
